:020000040000FA
:020000000528D1
:08000800212807309F0085014B
:10001000860183160E308500003086000230810094
:10002000831281018530A100A201A0308B00A208BB
:1000300003191B28172805140B11C0308100A20AD0
:1000400017288B12A400030EA3002208013A0319FB
:1000500032282208023A031936282208033A0319E3
:100060003F28592821088100A20A59280510831623
:10007000073081008312F9308100A20A59288316C3
:10008000023081008312A201851C4B28051D5328D4
:10009000851D4E2859288530A1005928A10803192B
:1000A0005228A1035928FF30210603195828A10A14
:1000B00059280B11230E8300A40E240E8B16090061
:02400E00503F21
:00000001FF
